:100000000C9434000C9451000C9451000C94510049
:100010000C9451000C9451000C9451000C942A0142
:100020000C9451000C9451000C9451000C94F90064
:100030000C9451000C9451000C94C8000C94510085
:100040000C9451000C9451000C9451000C945100EC
:100050000C9451000C9451000C9451000C945100DC
:100060000C9451000C94510011241FBECFEFD8E026
:10007000DEBFCDBF11E0A0E0B1E0E4EFF6E002C0EA
:1000800005900D92A031B107D9F711E0A0E1B1E0E0
:1000900001C01D92A531B107E1F70E9478010C94CF
:1000A00078030C940000CF92DF92EF92FF920F93AF
:1000B0001F93CF93DF93EC01C880D980EA80FB8047
:1000C00020E030E040E05FE3C701B6010E94F102AA
:1000D0000E9449029B01AC010E94A8019B01AC0156
:1000E000C701B6010E94A70101E010E020E030E066
:1000F00040E85FE30E94ED0287FF02C000E010E0ED
:100100001D830C838E859F858230910561F083303D
:10011000910599F00197C9F416BC80916E00826038
:1001200080936E0016C0109285001092840080911A
:100130006F00826080936F000CC01092B2008091BB
:10014000700082608093700004C081E090E00E94A3
:10015000780378949FB7F894809112019FBF882309
:10016000C9F310921201EA85FB858C819D81892B50
:1001700019F08081806202C080818F7D8083DF9151
:10018000CF911F910F91FF90EF90DF90CF90089546
:100190001F920F920FB60F9211242F933F938F93BC
:1001A0009F938091100190911101019690931101FC
:1001B0008093100180911201813091F02091100103
:1001C0003091110180911301909114012817390782
:1001D00038F081E080931201109211011092100109
:1001E0009F918F913F912F910F900FBE0F901F9075
:1001F00018951F920F920FB60F9211242F933F93D1
:100200008F939F938091100190911101019690938B
:1002100011018093100180911201813091F02091A1
:100220001001309111018091130190911401281750
:10023000390738F081E08093120110921101109279
:1002400010019F918F913F912F910F900FBE0F90B2
:100250001F9018951F920F920FB60F9211242F9393
:100260003F938F939F93809110019091110101967C
:10027000909311018093100180911201813091F0CF
:10028000209110013091110180911301909114017E
:100290002817390738F081E080931201109211017C
:1002A000109210019F918F913F912F910F900FBE4F
:1002B0000F901F901895FC0185B5836085BD21E0E6
:1002C00030E0358724878AE090E090931401809392
:1002D000130184B5826084BD89EF87BD3787268787
:1002E000259A85E290E09387828780E090E00895E8
:1002F000CF92DF92EF92FF9280E091E00E945B014B
:10030000C12CD12C760160E070E0CB01609300013C
:1003100070930101809302019093030180E091E0CA
:100320000E9453008FEFC81AD80AE80AF80AC701DA
:10033000B6010E940C022FE632E143E05BE30E942B
:10034000F10220E030E0A9010E94A801DFCF50585F
:10035000BB27AA270ED0F0C0E1D030F0E6D020F0C5
:1003600031F49F3F11F41EF4D6C00EF4E095E7FB84
:10037000A3C0E92FF2D080F3BA176207730784078E
:10038000950718F071F49EF521C10EF4E0950B2E3F
:10039000BA2FA02D0B01B90190010C01CA01A001D7
:1003A0001124FF27591B99F0593F50F4503E68F132
:1003B0001A16F040A22F232F342F4427585FF3CF73
:1003C000469537952795A795F0405395C9F77EF444
:1003D0001F16BA0B620B730B840BBAF09150A1F08D
:1003E000FF0FBB1F661F771F881FC2F70EC0BA0F13
:1003F000621F731F841F48F4879577956795B7959B
:10040000F7959E3F08F0B3CF9395880F08F0992792
:10041000EE0F979587950895E89409C097FB3EF4F1
:1004200090958095709561957F4F8F4F9F4F992341
:10043000A9F0F92F96E9BB279395F69587957795BF
:100440006795B795F111F8CFFAF4BB0F11F460FF7F
:100450001BC06F5F7F4F8F4F9F4F16C0882311F0D7
:1004600096E911C0772321F09EE8872F762F05C0EB
:10047000662371F096E8862F70E060E02AF09A9586
:10048000660F771F881FDAF7880F9695879597F97B
:10049000089585D080F09F3740F491110EF097C0F9
:1004A00060E070E080E89FEB089526F41B16611D64
:1004B000711D811D07C021C097F99F6780E870E01A
:1004C00060E00895882371F4772321F09850872BFA
:1004D000762F07C0662311F499270DC09051862B03
:1004E00070E060E02AF09A95660F771F881FDAF7B0
:1004F000880F9695879597F908959F3F31F0915011
:1005000020F4879577956795B795880F911D9695F7
:10051000879597F908959FEF80EC089500240A9439
:100520001616170618060906089500240A941216CE
:100530001306140605060895092E0394000C11F401
:10054000882352F0BB0F40F4BF2B11F460FF04C0AE
:100550006F5F7F4F8F4F9F4F089557FD9058440F07
:10056000551F59F05F3F71F04795880F97FB991F12
:1005700061F09F3F79F087950895121613061406CF
:10058000551FF2CF4695F1DF08C01616170618065C
:10059000991FF1CF86957105610508940895E5DFEF
:1005A000A0F0BEE7B91788F4BB279F3860F4161691
:1005B000B11D672F782F8827985FF7CF869577959D
:1005C0006795B11D93959639C8F30895E894BB27B4
:1005D00066277727CB0197F9089566D008F48FEF47
:1005E00008950BD0A9CF9ADF28F09FDF18F095234C
:1005F00009F062CF90CF1124EACFAFDFA0F3959F2F
:10060000D1F3950F50E0551F629FF001729FBB27F9
:10061000F00DB11D639FAA27F00DB11DAA1F649FA5
:100620006627B00DA11D661F829F2227B00DA11D58
:10063000621F739FB00DA11D621F839FA00D611DDE
:10064000221F749F3327A00D611D231F849F600DFF
:10065000211D822F762F6A2F11249F5750408AF038
:10066000E1F088234AF0EE0FFF1FBB1F661F771FC4
:10067000881F91505040A9F79E3F510570F01CCF44
:10068000A6CF5F3FECF3983EDCF3869577956795B0
:10069000B795F795E7959F5FC1F7FE2B880F911DE2
:1006A0009695879597F90895990F0008550FAA0B0D
:1006B000E0E8FEEF16161706E807F907C0F0121675
:1006C0001306E407F50798F0621B730B840B950B78
:1006D00039F40A2661F0232B242B252B21F40895CD
:1006E0000A2609F4A140A6958FEF811D811D08956A
:0406F000F894FFCFAC
:1006F4000000000000000AD7233C000000000000B6
:00000001FF
